:100000000C9496010C94BE010C94BE010C94BE019C
:100010000C94BE010C94BE010C94BE010C94BE0164
:100020000C94BE010C9467020C94E2210C945A22A9
:100030000C94BE010C94BE010C94BE010C94BE0144
:100040000C9410070C94BE010C94BE010C94BE01DC
:100050000C94BE010C94BE010C94BE010C948B193F
:100060000C94BE010C94211E0C945C1E0C94BE01D9
:100070000C94BE010C94BE010C94BE010C94BE0104
:100080000C94BE010C94BE010C94BE010C94BE01F4
:100090000C94BE010C94BE010C94BE010C94BE01E4
:1000A0000C94BE010C94BE010C94BE01D41AD71A54
:1000B000CA1ACE1AF81AF81AF81ADB1ADF1AE31A53
:1000C000E91AED1AF81AF31A434C49206E6F74209E
:1000D000617661696C61626C652C20757365206363
:1000E0006F6E666967757261746F7221000000003F
:1000F00000240027002A002D003000000000002509
:100100000028002B002E00310000000000230026F4
:100110000029002C002F0004040404040304050239
:100120000202020403020202020606060606060492
:100130000402020204040802011040804010204022
:1001400080408008020401804020100201108010CD
:100150002040400000000200080E000003040100DF
:100160000B00000000000000000000000000000084
:1001700000070605040100080A0B0C0D09080B0016
:10018000020202010009040000010202000005242D
:1001900000100105240101010424020605240600C3
:1001A000010705810310004009040100020A000054
:1001B000000705020240000007058302400000041A
:1001C0000309042203410072006400750069006E97
:1001D000006F0020004C0065006F006E006100722F
:1001E0000064006F0018034100720064007500692C
:1001F000006E006F0020004C004C00430012010014
:10020000020000004041233680000101020001127B
:10021000010002020000404123368000010102007B
:100220000100C18081C105010902A1010901A100EC
:10023000850105091901290315002501950375019B
:1002400081029501750581030501093009310938DD
:100250001581257F750895038106C0C00501090633
:10026000A1018502050719E029E71500250175019F
:10027000950881029501750881039506750815009A
:1002800025650507190029658100C00904020001E0
:100290000300000009210101000122650007058417
:1002A0000340000100000000000000002A2B28008D
:1002B000000000000000000000000000000000003E
:1002C000000000002C9EB4A0A1A2A434A6A7A5AE55
:1002D000362D3738271E1F20212223242526B3330D
:1002E000B62EB7B89F8485868788898A8B8C8D8E39
:1002F0008F909192939495969798999A9B9C9D2F05
:100300003130A3AD350405060708090A0B0C0D0EA4
:100310000F101112131415161718191A1B1C1DAFE4
:10032000B1B0B500A71B04204021C82311241FBE73
:10033000CFEFDAE0DEBFCDBF12E0A0E0B1E0E0E158
:10034000FBE402C005900D92A632B107D9F714E084
:10035000A6E2B2E001C01D92A33EB107E1F713E0AF
:10036000CCE2D3E004C02297FE010E946E25C43285
:10037000D107C9F70E9449200C9486250C940000EF
:10038000A0E0B0E0E6ECF1E00C943D25EC01A880A3
:10039000B980CA80DB80A114B104C104D10441F446
:1003A00084E2A82E89EDB82E8BE5C82E87E0D82EE2
:1003B000C601B5012DE133EF41E050E00E941A255E
:1003C00027EA31E440E050E00E94C6247B018C0122
:1003D000C601B5012DE133EF41E050E00E941A253E
:1003E000CA01B9012CEE34EF4FEF5FEF0E94C62433
:1003F0006E0D7F1D801F911F97FF04C061507040DC
:1004000080409048688379838A839B839B01AC01F9
:100410005F77B901CA01CDB7DEB7EAE00C94592580
:100420000E94C001089587E491E00E94C0010895F0
:1004300060934701709348018093490190934A016A
:10044000089580912602813019F482E0809326027B
:1004500080912602833019F484E080932602089567
:10046000009721F19C0140E050E068E478EE81E0E3
:1004700090E00E941A25C901DA018F3F9105A1057C
:10048000B10531F028F08FEF90E0A0E0B0E008C0B7
:100490000097A105B10521F481E090E0A0E0B0E073
:1004A0008093D1008091C000806103C08091C00022
:1004B0008F7E8093C0000895EBE6F0E08081806835
:1004C0008083E8E6F0E080818160808308951F9258
:1004D0000F920FB60F9211242F933F934F935F9378
:1004E0006F937F938F939F93AF93BF93EF93FF93FC
:1004F0001F9902C00E942102FF91EF91BF91AF911D
:100500009F918F917F916F915F914F913F912F912B
:100510000F900FBE0F901F90189581E008951F93C4
:10052000182F0E948D028823E9F02FB781E0809375
:10053000C703F89480910008909101088757974766
:1005400009F0A89588E18093600010936000112362
:1005500041F080910008909101088757974709F072
:10056000A8952FBF1F910895382F20E0809159033F
:1005700090915A038227932740E061E270E19C0149
:10058000220F331F97FF04C0C9018627972701C098
:10059000C9014F5F483099F790935A0380935903EC
:1005A000089587E380935C0280E092ECA1E0B0E0E4
:1005B00080935D0290935E02A0935F02B09360020D
:1005C00087E08093690280EC92E9ADEEB9E1809317
:1005D000610290936202A0936302B093640285E08B
:1005E00080936A028DEE9EEFADEABEED80936502C8
:1005F00090936602A0936702B0936802ABE6B2E004
:1006000080E090E0863010F0E0E004C0FC01E051B2
:10061000FE4FE081ED9301968831910599F782E0D4
:10062000809383028AE080938402089580EC91EDA8
:10063000A8E9BBE18093290290932A02A0932B02A0
:10064000B0932C0280E090E0A0E0B0E580932D0212
:1006500090932E02A0932F02B0933002E1E3F2E0D8
:1006600080E081938F5F8031E1F70895DC019896F7
:10067000EC91F0E0E770F070E851FE4F8081089552
:100680008F929F92AF92BF92CF92DF92EF92FF92A2
:100690000F931F938C010E943603D80197962C91DB
:1006A00030E043E150E0249FF001259FF00D349F9E
:1006B000F00D1124E55BFE4F80809180A280B38015
:1006C00090E00F96AA2797FDA095BA2FBC01CD0107
:1006D00020E43FE14DE750E00E94C624A5019401CB
:1006E0000E94F82469017A0180ED97E0A0E0B0E073
:1006F000C80ED91EEA1EFB1ED80198968C918871EF
:1007000081F060E07EEE8AEB9BE0A50194010E94FF
:10071000F82428513C4F4F4F5F4FC20ED31EE41EAA
:10072000F51E87EE93E0A0E0B0E0C80ED91EEA1EE9
:10073000FB1EC701B60128EE33E040E050E00E9406
:10074000F824CA01B90128EE33E040E050E00E94ED
:10075000C6241F910F91FF90EF90DF90CF90BF9034
:10076000AF909F908F9008958F3F910509F010F4FE
:1007700080E0089522E08030920710F481E008952F
:100780008050934010F083E0089582E00895CF9266
:10079000DF92FF920F931F93CF93DF93F82FEB011C
:1007A0006A01182F1695E0E088819981D6018C9313
:1007B0008A819B8111968C9311978C819D811296D1
:1007C0008C9312978E819F8113968C931397288117
:1007D00039814A815B816C817D818E819F81929577
:1007E000990F990F907C832F8370982B852F83709E
:1007F000880F880F982B872F83708295807F982B86
:1008000014969C9385E090E0C80ED91E2896EF5F61
:100810001E1750F6F0FF21C0888199810E94B40311
:10082000F82E8A819B810E94B403182F8C819D81B0
:100830000E94B403082F8E819F810E94B403F2941A
:10084000FF0CFF0C70ECF7221295107F1F29182B5C
:10085000000F000F012BD6010C93DF91CF911F9158
:100860000F91FF90DF90CF90089523E080329207A0
:1008700018F420E030E026C023E0883E920748F4D8
:100880009C012F51334054E0369527955A95E1F756
:1008900019C027E0803D920720F49C012C5D334075
:1008A00011C028E08839920718F02FEF33E00AC012
:1008B0009C01285C374044E0369527954A95E1F73E
:1008C0002D503C4FC90108958C30910548F49C018E
:1008D00074E0220F331F7A95E1F7285D3C4F17C073
:1008E00023E0843F920720F49C0124523C4F0FC028
:1008F00024E08030920718F020E938E008C09C011D
:100900002657334F64E0220F331F6A95E1F7C90180
:1009100008959C013695279525753575821B930B97
:100920009C013695279536952795237333738373EA
:100930009373280F391FC901E4E096958795EA95CE
:10094000E1F7820F931F8F709F7021E031E0AC01BF
:10095000429FC001439F900D529F900D1124892FFB
:100960000895882339F0299800002A9A0000299ACE
:1009700000000895299800002A980000299A000094
:100980000895299A000083B12998000090E0B3E00F
:1009900096958795BA95E1F7817008950F931F9307
:1009A000082F5E9A29985E9810E0802F80780E9428
:1009B000B104000F1F5F1830C1F729981F910F91E4
:1009C00008958F770E94CE0408950F931F93082FE8
:1009D00010E0802F80780E94B104000F1F5F183054
:1009E000C1F729981F910F9108950F931F9329988C
:1009F00080E000E0182F110F0E94C104810F0F5FEB
:100A00000830C1F71F910F9108950E94E1040E94E0
:100A1000F5045E9A08951F93162F80680E94CE04F5
:100A2000812F0E94E5045E9A1F9108951F931091F3
:100A300065021827ECE5F2E0E80FF11D89E767850C
:100A40000E940B058DE3612F0E940B0582E4612F4C
:100A50000E940B051F91089586E20E9405050895E6
:100A60000F931F938C018CE1F80164810E940B05A8
:100A70008DE1F80165810E940B058EE1F801668128
:100A80000E940B0580E2F80167810E940B0581E25C
:100A9000F80160850E940B0582E2F80161850E94E1
:100AA0000B0583E2F80162850E940B0584E2F801E0
:100AB00063850E940B0585E2F80164850E940B05A1
:100AC0008AE2F80165850E940B058EE6F8016685CD
:100AD0000E940B058FE6F80167850E940B0580E7F1
:100AE000F80160890E940B0581E7F80161890E9485
:100AF0000B0582E7F80162890E940B051F910F9197
:100B00000895EF92FF920F931F93CF93DF937B0192
:100B10008C01603028E372072CE982072CE19207F0
:100B200028F520E836E948E950E00E94F824E90178
:100B30006897B90180E090E020E839E647E65FEF8A
:100B40000E94C6246E0D7F1D801F911F32E0660F2C
:100B5000771F881F991F3A95D1F721E732E040E0CF
:100B600050E00E94F824890180E421C020E03DE2A9
:100B700041E351E00E94F824E9016897B90180E05F
:100B800090E020E033ED4EEC5EEF0E94C6246E0D47
:100B90007F1D801F911F660F771F881F991F21E7F8
:100BA00032E040E050E00E94F824890180E69E0196
:100BB0002F71622F680F85E70E940B0586E7612F72
:100BC0000E940B0587E7602F0E940B05CDB7DEB7AB
:100BD000E6E00C945D25682F8DE60E940B050895D4
:100BE0009F92AF92BF92CF92DF920F93DF93CF93FA
:100BF00000D000D0CDB7DEB7982E83E00E94050567
:100C00008093850284E00E9405058093860286E039
:100C100060E00E940B0587E061E00E940B0589E01F
:100C20006FE70E940B058AE065E00E940B058BE0F0
:100C300065E10E940B058CE062E10E940B058DE0EE
:100C40006DEF0E940B058EE060E00E940B0599207D
:100C500019F08AEA91E008C08091830223E1829F23
:100C6000C0011124855B9E4F0E94300580E36CE833
:100C70000E940B0582E36FE00E940B0583E362E4B0
:100C80000E940B0584E36AE00E940B0585E36AE29B
:100C90000E940B0586E36DE20E940B0587E364ED7D
:100CA0000E940B0588E360E00E940B0589E360E089
:100CB0000E940B05992049F065E8A62E61ECB62E3E
:100CC00061ECC62E6EEDD62E08C0A0906502B090E5
:100CD0006602C0906702D09068020AE38D2D9927C2
:100CE000AA27BB2789839A83AB83BC83802F698122
:100CF0000E940B05802F8B5F69810E940B05DC2C05
:100D0000CB2CBA2CAA240F5F0E3341F783E46FEF8C
:100D10000E940B0584E46FEF0E940B0585E46FEFE2
:100D20000E940B0586E46FEF0E940B05992019F0D5
:100D30008DE666E003C08DE6609169020E940B05B6
:100D400089E760E00E940B058AE760916A020E94D1
:100D50000B0583E760E00E940B0584E760E00E94DA
:100D60000B05992029F060EC72E98DEE99E108C03D
:100D700060916102709162028091630290916402BD
:100D80000E9481050F900F900F900F90CF91DF91EF
:100D90000F91DF90CF90BF90AF909F90089587E024
:100DA00061E00E940B058EE764E20E940B0588E07B
:100DB00063E00E940B0588E060E00E940B0587E07D
:100DC00065E00E940B0585E062E00E940B0583E070
:100DD0000E9405058093850284E00E9405058093AA
:100DE00086020895582F4091C202842F90E0FC01A2
:100DF000EF70F0709F012F5F3F4F74E095958795DE
:100E00007A95E1F72817390751F0EE54FD4F5083DA
:100E1000842F8F5F8F70407F842B8093C202089550
:100E20001F920F920FB60F9211241F932F933F938F
:100E30004F935F936F937F938F939F93AF93BF93E2
:100E4000CF93DF93EF93FF93C0918600D0918700FB
:100E500020910603309107038091E502882309F071
:100E600062C0BE01621B730B20912D0230912E02D5
:100E700040912F025091300225FD02C07695679572
:100E800089E0653C7807B8F18091DD011CE1569559
:100E90004795379527951A95D1F7211531054105C5
:100EA000510521F421E030E040E050E090E0A0E086
:100EB000B0E0281739074A075B07D0F48091DD01BD
:100EC0008F3FB1F020E00EC0E22FF0E0EE0FFF1FE9
:100ED000DF01AA51BD4F8D919C91E354FE4F918348
:100EE00080832F5F8091DD01281770F31092E40258
:100EF0001092DD0118C082E06D3B780760F18091AF
:100F0000DD01803140F51091DD01CB010E943504F7
:100F1000E12FF0E0EE0FFF1FEA51FD4F9183808338
:100F20001F5F1093DD01D0930703C0930603FF9169
:100F3000EF91DF91CF91BF91AF919F918F917F9171
:100F40006F915F914F913F912F911F910F900FBE25
:100F50000F901F9018958FEF8093DD01E4CF83E011
:100F6000809380008AE98093810080912D0286FD24
:100F700005C0809181008064809381008FEF9FEF96
:100F8000909389008093880080916F0080628093A5
:100F90006F0008956F3018F086958058089589E0A5
:100FA000689F802D11240895A0E0B0E0EAEDF7E0FD
:100FB0000C943F25182F0E94E1199B01AC018091F0
:100FC000530390915403A0915503B09156036901C6
:100FD0007A01C81AD90AEA0AFB0AD701C601895858
:100FE0009341A040B04010F010925203209353035D
:100FF0003093540340935503509356032091E502D8
:10100000822F81508230E8F580915203882309F4C1
:101010004FC1813011F482E0BCC1803108F035C18C
:10102000E82FF0E0EA51FD4F10838F5F8093520369
:10103000803109F0B0C1A8EEB2E0213039F4119648
:10104000EC911197E695E6958C9109C08D919C9154
:101050001197E92FE695E695E69596958795E03107
:1010600040F4F0E090E0EE0FFF1FE354FE4F918359
:1010700080831092E402129682E0A63FB807E9F658
:101080008AC1233009F004C180915203882321F4DE
:101090001F3009F080C10CC1883130F4E82FF0E036
:1010A000EB51FD4F108374C1883109F0EEC011235C
:1010B00009F0EBC0C0E0D0E00BE010E0DE0163E03F
:1010C000AA0FBB1F6A95E1F7C09FB001C19F700DC9
:1010D000D09F700D1124FB01EA51FD4F80812181C9
:1010E000922F977095958795FD01EE0FFF1FE354A2
:1010F000FE4F91838083FB01E951FD4F308136958E
:10110000369536952181422F4295440F407E842F9B
:10111000832B269526952695922F977095958795E2
:10112000FD01EE0FFF1FE154FE4F91838083FB0111
:10113000E851FD4F80818295869586958370418127
:10114000942F990F990F292F282B42954695469554
:10115000437082818170880F880F382F342B35952A
:101160002795FD01EE0FFF1FEF53FE4F31832083C4
:10117000FB01E651FD4F308136952181422F479585
:1011800044274795842F832B2695922F977095950A
:101190008795FD01EE0FFF1FED53FE4F9183808376
:1011A000FB01E551FD4F308132953F702181422F87
:1011B0004295407F842F832B22952F70922F97701A
:1011C00095958795FD01EE0FFF1FEB53FE4F918321
:1011D0008083FB01E451FD4F8081881F8827881F91
:1011E0004181942F990F292F282B441F4427441FF6
:1011F00082818370880F382F342B35952795FD0118
:10120000EE0FFF1FE953FE4F31832083FB01E251B4
:10121000FD4F3081369536952181422F4295440FFE
:10122000440F407C842F832B26952695922F977010
:1012300095958795AA0FBB1FFD01E753FE4F91833C
:10124000808361517D4FFB01208122952695277077
:101250004181342F330F330F330F832F822B942F81
:1012600092959695977095958795A553BE4F119633
:101270009C938E932196C230D10509F01FCF8091A7
:10128000FC0283FD02C01092E4021092520383C05C
:10129000243009F080C040915203442359F4183A95
:1012A000B1F410925A031092590388EA0E94B402D2
:1012B00081E06FC0413019F41093570304C04230ED
:1012C00031F410935803812F0E94B4025DC06091E5
:1012D0005803262F30E0220F331FE42FF0E0C9011E
:1012E00002968E179F0734F0433268F7ED51FD4F99
:1012F0001083E9CF2D5F3F4F4091590350915A031E
:10130000E217F30749F4912F80E0482759275093BB
:101310005A034093590338C0812F90E0481759076A
:1013200089F580915703813069F5613118F080E1CA
:1013300080935803D090580346EEE42E42E0F42EFA
:1013400000E010E01BC0F701D081C0E0818190E097
:101350008C2B9D2B33E0969587953A95E1F70E946B
:101360003504F801EE0FFF1FE354FE4F9183808395
:101370000F5F1F4F82E090E0E80EF91E0D1518F385
:101380001092E4021092520380915203882319F0C4
:101390008F5F80935203CDB7DEB7E8E00C945B25F6
:1013A000FF920F931F93CF93DF93182F092FF62EE1
:1013B0008EE30E940B05212F302FC901EC0110E0B4
:1013C00005C08FE769910E940B051F5F1F15C8F3C9
:1013D00085E064E00E940B0583E00E940505809390
:1013E000850284E00E940505809386020E94E1192F
:1013F00060938702709388028093890290938A0297
:1014000087E069E00E940B0581E080932602CDB75A
:10141000DEB7E5E00C945E250E94D009809126029B
:101420008130D9F40E94E11920918702309188021D
:101430004091890250918A02621B730B840B950BB9
:10144000605A76488140904040F4E8CF85E194E0CE
:1014500060E071E00E940C1E0895809126028130A8
:10146000A9F308958BEA94E06EE70E94C41F0895E3
:10147000A0E0B0E0EEE3FAE00C943E256C018BEACC
:1014800094E06EE70E94C41F760100E010E0C0E027
:10149000D0E0B0E2BB2E0AC00830110521F49E0155
:1014A0002095F60120870894E11CF11CF70160816A
:1014B000862F8D57823040F48BEA94E06DE70E94CE
:1014C000C41FF70160816B258BEA94E00E94C41F62
:1014D0000115110551F0F70180819E01280F311D82
:1014E000C32FDD27C20FD31FD0700F5F1F4F0930EE
:1014F000110591F6CDB7DEB7E9E00C945A25A9E0C5
:10150000B0E0E5E8FAE00C944525382FE62F80910D
:10151000C70290E0019664E270E00E94E524982FF3
:101520008093C70288E9898380E18A83913071F0D2
:10153000913028F0923099F09330E1F416C085E0B4
:101540008B8381EF8C832F5F2D8317C09B8381EF6B
:101550008C8384E6489FC00111249D830EC084E0E3
:101560008B8381EF8C833D8308C09B8381EF8C83C9
:10157000ED8303C00E94320A04C0CE0101960E948E
:10158000380A2996E2E00C9461250F931F93CF93BC
:10159000DF93182F092F8BEA94E06EE70E94C41F97
:1015A000212F302FC901EC0110E000E288818D5716
:1015B000823040F48BEA94E06DE70E94C41F88817A
:1015C000802788838BEA94E069910E94C41F1F5F83
:1015D000193061F78BEA94E06EE70E94C41FDF9137
:1015E000CF911F910F910895A9E0B0E0EAEFFAE0E2
:1015F0000C944525382F8091C702882379F48EEF0B
:1016000089833A836B83842F90E0959587958C83AB
:101610002D83198618861F821E822FC04091C20218
:10162000842F90E09C012F70307054E09595879541
:101630005A95E1F78217930721F18DEF89831A827A
:101640001B82DE01149620E008C0EE54FD4F80811D
:101650008D93405F2F5F263069F0842F90E0FC016E
:1016600034E0F595E7953A95E1F78F709070E817BB
:10167000F90759F74093C2022A83CE0101960E94CE
:10168000C50A8091C70290E0019666E070E00E9472
:10169000E5248093C7022996E2E00C9461259F928D
:1016A000AF92BF92CF92DF92EF92FF920F931F9370
:1016B000B82EA62ED42EC22E902E0E94E1197B01A8
:1016C0008C018091B1022091C3023091C4024091FB
:1016D000C5025091C6028823B1F0D801C701821B10
:1016E000930BA40BB50B815E9E42A040B04020F14D
:1016F0002C2DDC1408F42D2D8B2D6A2D422F292D35
:101700000E947F0A11C0D801C701821B930BA40B52
:10171000B50B81539547A040B04070F08B2D6A2DDA
:101720004D2D2C2D0E94F40AE092C302F092C402C7
:101730000093C5021093C6021F910F91FF90EF9086
:10174000DF90CF90BF90AF909F900895E82FF0E08A
:10175000E85DFD4FE185E03158F4F894F0E0EE0FDC
:10176000FF1FE354FE4F0190F081E02D789413C0E9
:10177000E03129F0E13129F0E0E0F2E00CC082E054
:1017800001C083E00E942C1B892B19F4ECE0F0E0EF
:1017900002C0E4EFF3E0CF010895A0E2B0E0E3ED92
:1017A000FBE00C943D258CE00E940505882379F52B
:1017B00085E194E06CE071E00E940C1E5F9A80E08D
:1017C0000E94F0050E94CF065F9821C08BEA94E04A
:1017D0000E948B1F482F8091E502882321F0842FDF
:1017E0000E94D40714C080915003E82FF0E0319696
:1017F0009F012F713070319780914F0390E028172F
:10180000390729F0EA5DFC4F4083209350038BEAAF
:1018100094E00E94511F892BC9F68091E50288232C
:1018200039F40CC085E194E00E94841B0E94D40727
:1018300085E194E00E945D1B892BA1F7809126022F
:10184000843009F08EC00E94E1196093D402709335
:10185000D5028093D6029093D70261157105810558
:10186000910561F481E090E0A0E0B0E08093D402C3
:101870009093D502A093D602B093D7028091E00254
:101880009091E10281609093E1028093E00283E015
:10189000809326028FE70E94E1040DE113E00E948D
:1018A000F504F80181938F01F3E006321F07B9F7C1
:1018B0004091080380911D03282F30E0842F90E091
:1018C0008227932786FF40C080E44827409308037F
:1018D000C90188739070C89709F510E014C01F5FA4
:1018E00080918402E12FF0E084FF06C0E35EFC4FAC
:1018F00080810E94F20607C0E35EFC4F8BEA94E011
:1019000060810E94C41F212F30E080911D0390E070
:10191000877090708217930714F716C02F7330707A
:10192000232B91F480911E038093D80280911F0392
:101930008093DA02809120038093DB02809123035D
:101940008093E2021092E30280915103813019F4F6
:1019500082E08093510380915103833011F41092FF
:1019600051030E94E1195B016C018091DC029091AE
:10197000DD02A091DE02B091DF020097A105B10562
:10198000C9F086017501E81AF90A0A0B1B0BD80188
:10199000C701885B9B40A040B04060F00E942C05CE
:1019A0008093D9021092DC021092DD021092DE02C6
:1019B0001092DF028CE592E00E9440032091D00259
:1019C0003091D1024091D2025091D302860175012B
:1019D000E21AF30A040B150BE616F70608071907B7
:1019E00008F42BC1A092D002B092D102C092D202D0
:1019F000D092D302809100089091010887579747B1
:101A000009F0A8958091E4028830A0F080912D0221
:101A100090912E02A0912F02B0913002FCE1B69578
:101A2000A79597958795FA95D1F70097A105B105E8
:101A300009F0A2C18091E4028F5F8093E402E090FC
:101A4000D402F090D5020091D6021091D702E11491
:101A5000F1040105110511F18CE592E00E944003AB
:101A6000AE18BF08C00AD10A6A157B058C059D0512
:101A700088F480912D0284FD04C080ED97E00E94DF
:101A800030021092D4021092D5021092D602109217
:101A9000D70204C080E090E00E94300290910803D9
:101AA000907C909308030091500310914F0301170D
:101AB000B1F180915103823091F5905890930803D1
:101AC0008CE592E00E943603893010F048E002C0B5
:101AD000482F415030E013C03F5FA32FB0E0812F6B
:101AE00090E0FC01EA5DFC4F2081FD01E85FFC4FC6
:101AF0002083AA5BBC4F2C930196182F1F713417BB
:101B000010F4101749F710934F03832F895C9091BD
:101B10000803892B80930803309346031AC0209151
:101B200051032430D1F490914603E7E4F3E0A9E0B7
:101B3000B3E0292F30E02E0F3F1F02C081918D931B
:101B4000E217F307D9F7995C80910803982B9093DB
:101B5000080383E08093510336C08091CB0282302A
:101B600059F49160909308035F9A01E312E07E01BB
:101B70000894E11CF11C10C0909308035F98222385
:101B800019F481E08093510380915103833069F708
:101B900084E080935103E9CFF80181918F010E9485
:101BA000A60BF701819391937F01F2E001341F07A7
:101BB00099F7809184028770BE016F5F7F4F49E083
:101BC00053E00E94C703469A2091C9022223A1F044
:101BD00090916902992381F08091CA028F5F80936E
:101BE000CA028150821729F41092CA02892F8150AB
:101BF00001C0892F0E94EB058091C8020E94160542
:101C00008CE592E00E943603682F88E093E00E9402
:101C1000D009E091C802EF5FE093C802E83131F0EB
:101C2000F0E0E45AFD4F8785882339F41092C8020A
:101C300004C05F9A89E08093E402809184028871F5
:101C400071F180912602823051F58091E0029091ED
:101C5000E102880F991F9093E1028093E00283E0F4
:101C6000809326020E94CF060E94E1196093DC0255
:101C70007093DD028093DE029093DF02611571059F
:101C80008105910561F481E090E0A0E0B0E08093EF
:101C9000DC029093DD02A093DE02B093DF0280911C
:101CA000840284FF1EC08091E0029091E1028E7F49
:101CB0000E948904182F8091D8026091E2020E944C
:101CC000CA07082F8091D902612F0E94CA07282FC6
:101CD0008091DA026091DB02402F009127020E947E
:101CE0004F0B46988091CB028130D1F0813020F0AB
:101CF000823009F047C034C082E10E942C1B892B3E
:101D000009F040C081E08093CB020E94D319609318
:101D1000CC027093CD028093CE029093CF0232C05A
:101D200082E10E942C1B892B21F50E94D31920915E
:101D3000CC023091CD024091CE025091CF02621B75
:101D4000730B840B950B695E734080409040D0F01C
:101D500082E08093CB0280ED97E00E94300212C0B7
:101D600082E10E942C1B892B69F080E090E00E94A8
:101D700030021092CB0206C08091E402883009F054
:101D800059CF57CFA096EAE00C945925219A229A70
:101D900023988BE060E00E94811A8CE061E00E9451
:101DA000811A089588E08093C1008AE061E00E9472
:101DB000811A8AE060E00E94F91A0895ACE1B0E06F
:101DC000E4EEFEE00C943D250E94E1197B018C01BC
:101DD00081E00E94F00584E7A82E6E010894C11CE2
:101DE000D11CB3E0BB2EA982C60161E00E940C0A9F
:101DF000B09226020E94CF066AEF70E080E090E089
:101E00000E94071A80912602833009F07DC085E187
:101E100094E00E945D1B892B09F076C00E94E119B5
:101E20006E197F09800B910B6058734C894C91405F
:101E300008F06AC0D8CF8FE70E94E1040E94F50441
:101E4000843509F05CC089830E94F504182F00E0F6
:101E50001093B0020093AF020E94F504080F111D09
:101E60001093B0020093AF020E94F5048093AE027B
:101E70000E94F5048093AD02813108F040C0FF2438
:101E800007C00E94F50403571D4FF8018083F394A7
:101E90000F2D10E08091AD0290E0880F991F081778
:101EA000190778F380E78983CE01019661E00E94EB
:101EB0000C0A83E0809326020E94CF0662E370E062
:101EC00080E090E00E94071A809126028330A9F0FA
:101ED0008FE70E94E1040E94F504803581F4898334
:101EE00001E412E00E94F504F80181938F01F2E011
:101EF0000C351F07B9F781E003C082E001C083E021
:101F00006C96EAE00C94592580912602833009F002
:101F100092CFF3CF83E00E9405058093850284E091
:101F20000E9405058093860287E061E00E940B0510
:101F30006AE070E080E090E00E94071A0E94CF06FD
:101F4000000008950F931F93082F17C05F9A64E64F
:101F500070E080E090E00E94071A5F9864E670E00D
:101F600080E090E00E94071A1F5F101778F36CE280
:101F700071E080E090E00E94071A10E0F6CF482F51
:101F8000392F25E00DC0F999FECF1FBA842F932F6A
:101F900092BD81BD60BD0FB6F894FA9AF99A0FBE52
:101FA000215059F0F999FECF842F932F92BD81BD16
:101FB000F89A80B5681739F7089582E00E94A20F59
:101FC0000895A0E0B0E0E7EEFFE00C943625482E3F
:101FD000562EEE24FF2488249924C0E0D0E0CC249F
:101FE000DD2476E4372E04C055245394CC24DD241C
:101FF000442069F480912702839DE001112468E266
:10200000E62E62E0F62E59E1852E912C1DC021E0CE
:10201000421671F480912702839DE00111246B9692
:102020004CE5E42E42E0F42E39E2832E912C0CC0D4
:1020300032E0431649F427E2E22E22E0F22E91E04C
:10204000892E912CC8E1D1E03E016C0C7D1C1092D0
:102050005A0310925903E3011BC0552059F4F99912
:10206000FECFD2BDC1BDF89A80B5F701E00FF11FD8
:10207000808307C0F701E00FF11FCE0160810E944D
:10208000BF0F0E0D1F1DF80180810E94B402219622
:102090009E012619022F10E008151905F0F2CE0155
:1020A0005520D9F4F999FECFD2BDC1BDF89A20B51B
:1020B000F999FECF2196D2BDC1BD2197F89A80B57E
:1020C00090E0B22EAA248A299B29209159033091AD
:1020D0005A032817390759F487CF219660915A037C
:1020E0000E94BF0FCE01609159030E94BF0F80E292
:1020F00091E0C80ED91E91EEC91692E0D90608F4F7
:1021000077CF852DCDB7DEB7E1E10C94522580E085
:1021100061E00E94E10F81E061E00E94E10F08951B
:1021200082E061E00E94E10F089582E060E00E9499
:10213000E10F80912702843020F0109227020E9444
:10214000901008951F93182F0E94951080912702D8
:10215000811731F0143020F4109327020E94901060
:102160001F9108951F93182F0E94E1196093C302D5
:102170007093C4028093C5029093C6021093B1027B
:10218000112329F440E855E260E070E004C040E02B
:1021900051EE60E070E08BEA94E00E94CA1E1F914D
:1021A000089585E194E060918C020E94BE1B089521
:1021B0001F93182F85E194E0612F0E94BE1B809130
:1021C0008C02812780938C021F9108951F93192FF1
:1021D0000E94D810812F0E94D8101F910895DF927D
:1021E000EF92FF920F931F93D82E7B0110928C02D7
:1021F00005E114E0C80165EB0E94BE1BC80162E660
:102200000E94BE1B8D2D0E94D810C7010E94E610AF
:102210001F910F91FF90EF90DF900895EF92FF9242
:102220000F931F937C0105E114E0C8016F2D70E04E
:102230004AE050E00E94891DC8016EE20E94B41C71
:10224000B701E4E076956795EA95E1F76F707070F5
:10225000C8014AE050E00E94891DC8016EE20E9458
:10226000B41C8FE0E822FF24C801B7014AE050E027
:102270000E94891D1F910F91FF90EF900895A2E297
:10228000B0E0E5E4F1E10C9435258E010F5F1F4FBE
:1022900080E1D8011D928A95E9F785E194E06BE130
:1022A00071E00E940C1E0E948A0F20E431EE4DE97D
:1022B00058E12F8F38A349A35AA380EC91EDA8E9E8
:1022C000BBE18B8F9C8FAD8FBE8F24EF31E040E060
:1022D00050E02F8B388F498F5A8F80E5C82E83ECC2
:1022E000D82EE12CF12CB0E44B2EB1EE5B2EBDE9E3
:1022F0006B2EB8E17B2E88249924540133241E8A46
:102300001D8A198A1A8A1B8A1C8AFFC085E194E0FB
:102310000E94841B8434B9F0853430F48332B9F1DF
:102320008C3209F0CCC044C0833509F0C8C02F8D71
:1023300038A149A15AA1C901DA012C013D01882423
:1023400099245401E2C085E194E064E40E94B41C45
:1023500085E194E040E451EE6DE978E12AE030E077
:102360000E94AC1D85E194E06CE20E94B41C85E102
:1023700094E040EC51ED68E97BE12AE030E00E9416
:10238000AC1D85E194E06CE20E94E61CBEC019829F
:102390001A821B821C821D821E821F821886198649
:1023A0001A861B861C861D861E861F86188A3AC0C2
:1023B000339434E0331609F0A8C069817A818B81A7
:1023C0009C8128EE33E040E050E00E94C6246F8FED
:1023D00078A389A39AA36D817E818F8198850E94BD
:1023E000C6246B8F7C8F8D8F9E8F89859A85AB8558
:1023F000BC858F8B988FA98FBA8F6D857E858F85D1
:1024000098890E94C6246B017C0190E2C9169EE463
:10241000D90690E0E90690E0F90630F48CE162E339
:102420000E940B05332471C0A0E3CA16A5E7DA06A3
:10243000A0E0EA06A0E0FA0618F48CE162E2F0CF30
:10244000B0E4CB16BCE9DB06B0E0EB06B0E0FB067F
:1024500018F48CE166E2E4CFE0E5CE16E3ECDE06AC
:10246000E0E0EE06E0E0FE0618F48CE162E1D8CF91
:10247000F0E6CF16FAEEDF06F0E0EF06F0E0FF063A
:1024800018F48CE165E1CCCF20E7C21621E1D20639
:1024900021E0E20620E0F20618F48CE161E0C0CF12
:1024A00030EAC31636E8D30631E0E30630E0F3063F
:1024B00018F48CE163E0B4CF8CE165E0B1CFA0ED1E
:1024C0002A2E280E49E0421500F1032D10E0000FDE
:1024D000111F000F111F81E090E08C0F9D1F080F4E
:1024E000191FD8016D917D918D919C912AE030E06A
:1024F00040E050E00E94C624620D711D811D911DB7
:10250000F801608371838283938385E194E00E9464
:102510005D1B892B09F0FACE81149104A104B1044A
:1025200089F4C301B2010E94810561E070E080E09E
:1025300090E00E94071AFFEFFE8B1D8A198A1A8A03
:102540001B8A1C8A2F89388D498D5A8D82169306D5
:10255000A406B506E0F40E942C0529893A894B8926
:102560005C89280F311D411D511D298B3A8B4B8BE6
:102570005C8B3D89381708F48D8B4E89841708F4DD
:102580008E8B0894811C911CA11CB11C56C0C301E8
:10259000B20128EE33E040E050E00E94F82485E1EB
:1025A00094E0BA01A9012AE030E00E947A1D85E199
:1025B00094E06CE20E94B41C85E194E06D894AE0ED
:1025C00050E00E949A1D85E194E06CE20E94B41CE8
:1025D00069897A898B899C89A50194010E94F824D4
:1025E00085E194E0BA01A9012AE030E00E947A1D59
:1025F00085E194E06CE20E94B41C85E194E06E8970
:102600004AE050E00E949A1D85E194E06CE20E944D
:10261000E61C4C0C5D1C6E1C7F1C8B8D9C8DAD8D47
:10262000BE8D84159505A605B70520F44F8C58A0DE
:1026300069A07AA08824992454012F8D38A149A13A
:102640005AA1285E33404040504009F05ECFA29628
:10265000E2E10C945125A0E0B0E0E1E3F3E10C9459
:1026600040250E94E1196115710581059105C9F3A5
:102670000E94180210926502109266021092670280
:1026800010926802DD24E0906502F09066020091ED
:10269000670210916802102F0F2DFE2CEE240E946D
:1026A00013022FEF30E040E050E00E941A25E60EC2
:1026B000F71E081F191FE0926502F0926602009350
:1026C000670210936802D39444E0D416E1F6CBE697
:1026D000D2E000E010E090E1E92E97E2F92E4EC042
:1026E0000F5F19F40E94D1024DC00E94130222E331
:1026F00030E040E050E00E941A256F5FEBE6F2E028
:1027000090E004C08191861759F39F5F9117D0F331
:1027100080916A0290E08E9D90018F9D300D9E9D6C
:10272000300D1124862F90E0AC01249FC001259F1D
:10273000900D349F900D1124AA2797FDA095BA2FD4
:1027400020916102309162024091630250916402D3
:10275000820F931FA41FB51F2091290230912A02D6
:1027600040912B0250912C02281739074A075B072A
:1027700008F4B6CF69931F5F183121F08881882350
:1027800009F0AECFCDB7DEB7E7E00C945C2580E072
:1027900060E00E94E10F882331F081E060E00E9458
:1027A000E10F882341F40E9416030E94D1020E9487
:1027B0002B130E9487100895AAE5B0E0E2EEF3E142
:1027C0000C9441258B017A018B3009F425C18C30A2
:1027D00040F5853009F484C0863080F4823009F4F5
:1027E00059C0833020F4813009F04FC242C0833099
:1027F00009F461C0843009F048C265C0883009F42A
:102800009DC0893038F4863009F486C0873009F0DD
:102810003CC28CC0893009F499C08A3009F035C2B5
:10282000C9C0893609F481C18A3680F4863609F434
:102830002CC1873620F4853609F027C20DC18736B2
:1028400009F43CC1883609F020C240C18C3609F435
:10285000C3C18D3638F48A3609F472C18B3609F05B
:1028600014C2AEC18D3609F4EBC1873C09F00DC22C
:10287000FFC181E069E270E00E94EF100CE512E018
:10288000F80181918F010E94D810F2E005381F07EE
:10289000B9F703C282E06BE170E00E94EF1001E43F
:1028A00012E0F80181918F010E94D810F2E00C35FE
:1028B0001F07B9F7F2C183E061E070E00E94EF10FA
:1028C0000E94DE0EE8C184E061E070E00E94EF103B
:1028D00081E00E94D8100E94D1100E943F11DFC1F8
:1028E0006091AD0270E0660F771F85E00E94EF10E7
:1028F00000E010E008C0F801E357FD4F80810E941E
:10290000D8100F5F1F4F8091AD0290E0880F991F84
:102910000817190780F3C1C186E062E070E00E94E9
:10292000EF1083E793E00E94E610B7C187E061E013
:1029300070E00E94EF108091AE02ADC188E061E0CE
:1029400070E00E94EF1080912702A5C186E689837E
:10295000CE01019661E00E940C0A0E94CF0683E03E
:102960008093260268EC70E080E090E00E94071AF5
:10297000809126028430E1F48FE70E94E1040E94F6
:10298000F5048983863471F489E060E270E00E9486
:10299000EF1010E00E94F5040E94D8101F5F103263
:1029A000C9F77BC189E061E070E00E94EF10C6C00A
:1029B00089E06CC18AE069E170E00E94EF1010923A
:1029C00028028091C703882351F080912D029091B5
:1029D0002E02A0912F02B0913002806809C0809130
:1029E0002D0290912E02A0912F02B09130028F778C
:1029F00080932D0290932E02A0932F02B093300269
:102A000008E212E0F80181918F010E94D810F2E0F3
:102A100001341F07B9F741C18BE061E270E00E9409
:102A2000EF108091E4028F3F39F08091E4028F5FD4
:102A30008093E402815002C08091E4020E94D81089
:102A400010E0812F0E94A60B0E9464040E94E610F1
:102A50001F5F1031B1F721C185E661E070E00E948F
:102A6000EF100932110509F015C120E030E0F9013D
:102A7000E45AFD4FD701A20FB31F8C9180832F5FC3
:102A80003F4F2932310599F759C086E661E070E081
:102A90000E94EF100B31110509F0FCC020E030E07E
:102AA000F901EF5BFD4FD701A20FB31F8C9180831B
:102AB0002F5F3F4F2B31310599F740C087E661E02A
:102AC00070E00E94EF100E94871038C088E661E035
:102AD00070E00E94EF1085E78A83DE011396E1E43F
:102AE000F2E08BE101900D928150E1F7CE01029668
:102AF0006CE10E940C0A0E94CF0683E080932602BC
:102B000060E273E080E090E00E94071A8091260264
:102B1000843009F0BFC08FE70E94E1040E94F504F1
:102B20008A83853509F0B6C009C089E661E070E0A6
:102B30000E94EF100E94D1020E94160381E0ABC0F8
:102B40008AE661E070E00E94EF1089E68E8FCE0188
:102B50004E9661E00E940C0A0E94CF0683E08093AB
:102B6000260260E273E080E090E00E94071A809104
:102B70002602843009F08EC08FE70E94E1040E9493
:102B8000F5048E8F8E01015E1F4F3AE3E32EF12C88
:102B9000EC0EFD1E0E94F504F80181938F01EE15E5
:102BA000FF05C1F7A1E4B2E0FE017F968BE1019041
:102BB0000D928150E1F78E8D893409F06BC0BECF44
:102BC0008BE661E070E00E94EF10F70180810E94C7
:102BD000A2100E94C713B2CF8CE661E070E00E94A1
:102BE000EF100032110571F487E68AAFDE01DB9643
:102BF000F70180E201900D928150E1F7CE01CA9673
:102C000061E205C087E48AAFCE01CA9661E00E9406
:102C10000C0A0E94CF0683E0809326026CE474E0E5
:102C200080E090E00E94071A80912602843091F59E
:102C30008FE70E94E1040E94F504873459F57ECFA6
:102C40008DE661E070E00E94EF100931110511F589
:102C500020E030E0F901E85DFD4FD701A20FB31F7E
:102C60008C9180832F5F3F4F2931310599F766CFD3
:102C700087EC61E070E00E94EF1081E00E94D810C4
:102C80000E94D11010928B020AC08AEC61E070E0C1
:102C90000E94EF1080E00E94D8100E94D110C65A06
:102CA000DF4FE6E00C945D25A0E0B0E0EAE5F6E158
:102CB0000C943D25B4E0AB2EA6E0BA2EF5E0CF2E65
:102CC0000BE513E0E4E6DE2E72E0E72E63E0F62E7D
:102CD000A1C085E194E00E94841B982F8093C603D5
:102CE0008091C503833021F1843028F4813099F03C
:102CF0008230B8F409C0853009F448C0853020F12D
:102D0000863009F087C05FC0953B09F083C081E041
:102D10008093C5037FC0923609F07AC0E092C50364
:102D200079C09093C4039093C303F092C50372C01B
:102D30009093C1031092C2038091C30389278093AB
:102D4000C303A092C50366C0D92FC0E02091C10380
:102D50003091C2032C2B3D2B3093C2032093C1032F
:102D60008091C30389278093C303C092C50325368E
:102D7000310508F44FC08CEC61E070E00E94EF1068
:102D800081E00E94D8100E94D11042C02091BF0360
:102D90003091C003F901E55AFC4F90838091C30341
:102DA00089278093C3032F5F3F4F3093C003209345
:102DB000BF038091C1039091C2032817390750F1D6
:102DC000B092C50327C08091C303891759F460915D
:102DD000BF037091C0038091C4034BE553E00E9490
:102DE000DC130DC08BEC62E070E00E94EF1080916C
:102DF000C4030E94D81080918C020E94D810F80160
:102E00008D2D11928A95E9F71092C0031092BF039D
:102E10001092C50385E194E00E945D1B892B09F0A7
:102E200058CFCDB7DEB7EAE00C94592581E0809306
:102E30008B0208C085E194E00E945D1B892B11F094
:102E40000E94541680918B028823A1F70895AAE26C
:102E5000B0E0EDE2F7E10C943A250E94D3197B0132
:102E60008C0181E00E94F00504C085E194E00E949D
:102E7000841B85E194E00E945D1B892BB1F75F986C
:102E8000DD24D39422E6722E92E0892E912C8C0EB2
:102E90009D1E5E010894A11CB11C83E0C82E0E94F7
:102EA000D31920E030E06E197F09800B910B693C4B
:102EB00071058105910510F021E030E08D2D90E045
:102EC00028233923232B99F10E94D3197B018C01EC
:102ED000469A80ED97E00E9430027982D401ECE5B9
:102EE000F2E089E201900D928150E1F7C5016AE2BA
:102EF0000E940C0A469880E090E00E943002C09246
:102F000026020E94CF0662E370E080E090E00E941B
:102F1000071A80912602843051F4C09226028FE76E
:102F20000E94E1040E94F504823409F4DD2482E168
:102F30000E942C1B892B39F5DD24D39424C05F9A81
:102F4000469A85E194E00E94841B8D30910569F0DA
:102F50008E3091051CF40A97A1F407C083329105C5
:102F600059F08234910569F40AC085E194E068EC77
:102F700070E00E94D21C05C00E943F1102C00E9456
:102F800016175F98469885E194E00E945D1B892B97
:102F900009F485CFD4CF8F929F92AF92BF92CF92F8
:102FA000DF92EF92FF920F931F9382E10E942C1BFE
:102FB000892B09F083C068EC70E080E090E00E940B
:102FC000071A80E090E00E9430020E94D3195B0152
:102FD0006C0130ECE32E32E1F32E012D112DE60EC3
:102FE000F71E081F191F06C082E10E942C1B892BA7
:102FF00009F062C00E94D3196E157F058007910702
:1030000098F382E10E942C1B892B09F055C080EDBA
:1030100097E00E9430020E94D3197B018C01992411
:103020009394882488E496E2A0E0B0E0A80EB91E4C
:10303000CA1EDB1E29C0AE14BF04C006D10638F478
:1030400080ED97E00E943002882483941DC00E9486
:10305000D3196E197F09800B910B693C71058105AD
:10306000910590F00E94D3197B018C0180E099209A
:1030700009F481E0982E882319F480E090E002C0E2
:1030800080ED97E00E94300282E10E942C1B892B88
:1030900091F280E090E00E943002882049F0809117
:1030A00027028F5F83700E94A2100E94C71306C080
:1030B0000E942B130E9487100E9427171F910F91C7
:1030C000FF90EF90DF90CF90BF90AF909F908F9048
:1030D0000895EF92FF920F931F9380E00E948F025A
:1030E0000E94C60E86E061E00E94811A85E061E0E0
:1030F0000E94811A82E160E00E94811A84E060E00F
:103100000E94811A84E061E00E94F91A0E94D20EA6
:1031100085E194E060E070E00E945C1B0E949510E5
:103120000E94C7130E94AF078FEF8093E4020E94B2
:103130005C0278940E94D3197B018C018091E40297
:103140008F3F09F0DEC00E94D3196E197F09800BF2
:10315000910B605D77408040904008F0D2C0EECF88
:1031600085E194E00E94841B85E194E00E945D1B50
:10317000892BB1F785E194E068E271E00E94091EB5
:1031800083E793E00E940E1185E194E06FE371E024
:103190000E94091E85E194E066E070E04AE050E09C
:1031A0000E94F51D62E370E080E090E00E94071A43
:1031B00085E194E00E945D1B04970CF185E194E0A9
:1031C0000E94841B82349105D1F485E194E00E9431
:1031D000841B8E34910599F485E194E00E94841B50
:1031E0008434910561F485E194E00E94841B819709
:1031F00031F480E090E00E9430020E942717409155
:103200005D0250915E0260915F0270916002DB018D
:10321000CA010197A109B1090497A105B10568F494
:103220004093E502433029F040E052EC61E070E069
:1032300004C040EA56E861E070E08BEA94E00E9446
:10324000CA1E0E94CB175F9880E090E00E94300277
:103250000E94AF071092C90280912D0283FF11C016
:1032600080917102882351F080917802882331F097
:1032700080917F02882311F087E001C085E0809370
:10328000C90280E00E94F0058091C8020E941605E4
:103290000E94CF0610924F031092500310925103D8
:1032A00010E015C062E370E080E090E00E94071A31
:1032B00080ED97E00E94300262E370E080E090E0F1
:1032C0000E94071A80E090E00E9430021F5F809108
:1032D0002702811738F78091840290E084FF09C0AB
:1032E00020E088719070489709F421E0822F0E94B5
:1032F000B2108FE00E948F021F910F91FF90EF900C
:10330000089580ED97E00E94300282E161E00E9422
:10331000F91A5F9A29CF1F920F920FB60F921124BC
:103320002F933F938F939F93AF93BF938091CC0341
:103330009091CD03A091CE03B091CF033091D003F3
:103340000196A11DB11D232F2D5F2D3720F02D5784
:103350000196A11DB11D2093D0038093CC039093BF
:10336000CD03A093CE03B093CF038091C803909177
:10337000C903A091CA03B091CB030196A11DB11D51
:103380008093C8039093C903A093CA03B093CB035F
:10339000BF91AF919F918F913F912F910F900FBE51
:1033A0000F901F9018958FB7F8942091CC0330910F
:1033B000CD034091CE035091CF038FBFB901CA0115
:1033C00008959FB7F8942091C8033091C9034091A4
:1033D000CA035091CB0386B5A89B06C08F3F21F04E
:1033E0002F5F3F4F4F4F5F4F9FBF542F432F322FC1
:1033F0002227280F311D411D511D82E0220F331F4E
:10340000441F551F8A95D1F7B901CA010895EF925B
:10341000FF920F931F93CF93DF937B018C010E9448
:10342000E119EB010EC00E94E1196C1B7D0B685E77
:103430007340C8F30894E108F10801091109C85163
:10344000DC4FE114F1040105110569F7CDB7DEB7D2
:10345000E6E00C945D25789484B5826084BD84B5E3
:10346000816084BD85B5826085BD85B5816085BD7F
:10347000EEE6F0E0808181608083E1E8F0E0108298
:10348000808182608083808181608083E0E8F0E0D9
:10349000808181608083E1E9F0E0808182608083C7
:1034A000808181608083E0E9F0E0808181608083B9
:1034B000E1ECF0E0808184608083808182608083A1
:1034C000808181608083E3ECF0E080818160808393
:1034D000E0ECF0E0808182608083E2ECF0E08081CB
:1034E00081608083EAE7F0E080818460808380816E
:1034F0008260808380818160808380818068808316
:103500000895CF93DF93482F50E0CA018B5C9E4F04
:10351000FC013491495E5E4FFA018491882369F180
:1035200090E0880F991FFC01E351FF4FA591B491E2
:10353000FC01E550FF4FC591D491662351F42FB79C
:10354000F8948C91932F909589238C93888189236B
:103550000BC0623061F42FB7F8948C91932F909543
:1035600089238C938881832B88832FBF06C09FB7C4
:10357000F8948C91832B8C939FBFDF91CF9108950A
:1035800090E0FC013197EE30F10590F5EA5AFF4FDB
:103590000C946C25809180008F7703C0809180000F
:1035A0008F7D80938000089584B58F7702C084B5A5
:1035B0008F7D84BD0895809190008F7707C08091A2
:1035C00090008F7D03C080919000877F8093900052
:1035D00008958091C0008F7703C08091C0008F7DD7
:1035E0008093C00008958091C200877F8093C200BD
:1035F0000895FF920F931F93F62E482F50E0CA01B3
:103600008D5A9E4FFC012491CA018B5C9E4FFC0198
:103610001491495E5E4FFA0104910023C9F0222300
:1036200019F0822F0E94C01AE02FF0E0EE0FFF1F6A
:10363000E550FF4FA591B4919FB7F894FF2021F476
:103640008C911095812302C08C91812B8C939FBF0C
:103650001F910F91FF9008950F931F93482F50E0F3
:10366000CA018D5A9E4FFC012491CA018B5C9E4F6A
:10367000FC010491495E5E4FFA011491112319F483
:1036800020E030E015C0222319F0822F0E94C01ADA
:10369000812F90E0880F991F875F9E4FFC01A591B5
:1036A000B4918C9120E030E0802311F021E030E0F3
:1036B000C9011F910F91089508952091110430912F
:1036C00012048091130490911404281B390B2F735A
:1036D0003070C90108952091110430911204809135
:1036E0001304909114042817390719F42FEF3FEFB2
:1036F00009C0E0911304F0911404EF52FC4F808153
:10370000282F30E0C901089520911104309112044E
:1037100080911304909114042817390719F42FEF9E
:103720003FEF13C0E0911304F0911404EF52FC4FEB
:103730002081809113049091140401968F739070EE
:10374000909314048093130430E0C90108951092FB
:1037500018041092170488EE93E0A0E0B0E0809384
:10376000190490931A04A0931B04B0931C048AEFCD
:1037700091E090931604809315040895A1E0B0E0C1
:10378000E4ECFBE10C9443258C0169838091E50115
:10379000882369F083E0BE016F5F7F4F41E050E016
:1037A0000E945F211816190614F49C0107C081E0DD
:1037B00090E0F8019383828320E030E0C9012196F4
:1037C000E4E00C945F2583E00E9436210895CF93B6
:1037D000DF9312C082E00E94A6202FEF8F3F920756
:1037E000C9F0E0911104F0911204EF52FC4F808374
:1037F000D0931204C0931104C0911104D09112040B
:103800002196CF73D0708091130490911404C8173F
:10381000D90701F7DF91CF910895FC0180818E5F78
:10382000808380E86DE771E042E450E00E94DD2093
:103830000895FC0181819081913A59F4813209F017
:103840004CC080E06EED71E047E050E00E94DD206A
:1038500042C0913209F041C0803239F48EED91E0DE
:1038600067E070E00E94212136C0823209F035C045
:1038700082818093E5018091DE019091DF01A0912A
:10388000E001B091E101805B9440A040B04019F5A7
:103890008091E50180FD12C087E797E790930108CA
:1038A000809300082BE088E190E00FB6F894A8958B
:1038B000809360000FBE209360000DC088E10FB6BA
:1038C000F89480936000109260000FBEA89510924B
:1038D00001081092000881E0089580E00895A0E0BA
:1038E000B0E0E5E7FCE10C943F257C016B018A0127
:1038F000C0E0D0E00FC0D6016D916D01D701ED9110
:10390000FC910190F081E02DC7010995C80FD91FE6
:10391000015010400115110571F7CE01CDB7DEB78A
:10392000E8E00C945B25EF92FF920F931F93CF93E7
:10393000DF937C018B01C0E0D0E0F8010F5F1F4FE7
:103940006491662359F0D701ED91FC910190F081CB
:10395000E02DC7010995C80FD91FEFCFCE01CDB714
:10396000DEB7E6E00C945D25DC01ED91FC91019061
:10397000F081E02D09950895EF92FF920F931F9328
:103980008C016DE00E94B41C7C01C8016AE00E94B9
:10399000B41C9C012E0D3F1DC9011F910F91FF907A
:1039A000EF900895EF92FF920F931F937C010E9476
:1039B000931C8C01C7010E94BC1C9C01200F311F6D
:1039C000C9011F910F91FF90EF900895EF92FF9220
:1039D0000F931F937C010E94B41C8C01C7010E94AD
:1039E000BC1C9C01200F311FC9011F910F91FF903A
:1039F000EF900895CF93DF93EC016115710519F4F1
:103A000020E030E00FC0DB010D900020E9F71197B6
:103A1000A61BB70BE881F9810280F381E02DAD018F
:103A200009959C01C901DF91CF9108954F925F9252
:103A30007F928F929F92AF92BF92CF92DF92EF923E
:103A4000FF920F931F93DF93CF93CDB7DEB7A1976C
:103A50000FB6F894DEBF0FBECDBF2C01742ECB0184
:103A6000223008F42AE019A231E2C32ED12CCC0E68
:103A7000DD1E822E9924AA24BB24672D752FA50153
:103A800094010E94F82479018A01C801B701A501B7
:103A900094010E94C624472D461B0894C108D108F2
:103AA0004A3010F4405D01C0495CF6014083E114E6
:103AB000F1040105110521F07E2C5F2DC801DDCF39
:103AC000C201B6010E94FA1CA1960FB6F894DEBF9F
:103AD0000FBECDBFCF91DF911F910F91FF90EF905F
:103AE000DF90CF90BF90AF909F908F907F905F902E
:103AF0004F900895DC012115310541F4ED91FC91C1
:103B00000190F081E02D642F099508950E94161D03
:103B10000895EF92FF920F931F939A017B0100E0AB
:103B200010E0B801A7010E947A1D1F910F91FF902C
:103B3000EF900895EF92FF920F931F939A01E62E54
:103B4000FF2400E010E0B801A7010E947A1D1F9138
:103B50000F91FF90EF900895A0E0B0E0E2EBFDE15F
:103B60000C943F25EC016A017B012115310541F4DC
:103B7000E881F9810190F081E02D642F09951BC047
:103B80002A303105B1F477FF13C06DE20E94B41CF6
:103B90008C0144275527BA014C195D096E097F092C
:103BA000CE012AE00E94161D9C01200F311F04C087
:103BB0002AE00E94161D9C01C901CDB7DEB7E8E0DE
:103BC0000C945B25EF92FF920F931F937B019A0158
:103BD0000027F7FC0095102FB801A7010E94AC1D2B
:103BE0001F910F91FF90EF900895EF92FF920F9326
:103BF0001F937C010E94E21D8C01C7010E94BC1C26
:103C00009C01200F311FC9011F910F91FF90EF9070
:103C100008950E94FA1C0895EF92FF920F931F934C
:103C20007C010E94091E8C01C7010E94BC1C9C01E2
:103C3000200F311FC9011F910F91FF90EF90089540
:103C400008951F920F920FB60F9211242F933F9356
:103C50004F938F939F93EF93FF938091C80082FDC2
:103C60001DC04091CE0020916304309164042F5F09
:103C70003F4F2F7330708091650490916604281730
:103C8000390771F0E0916304F0916404ED5DFB4F3E
:103C90004083309364042093630402C08091CE007B
:103CA000FF91EF919F918F914F913F912F910F90A5
:103CB0000FBE0F901F9018951F920F920FB60F9284
:103CC00011242F933F938F939F93EF93FF93209112
:103CD000A7043091A8048091A9049091AA04281700
:103CE000390731F48091C9008F7D8093C90014C0D9
:103CF000E091A904F091AA04E959FB4F2081809139
:103D0000A9049091AA0401968F7390709093AA04CD
:103D10008093A9042093CE00FF91EF919F918F9102
:103D20003F912F910F900FBE0F901F901895A0E01C
:103D3000B0E0EDE9FEE10C943B25FC011382128218
:103D400088EE93E0A0E0B0E084839583A683B783F8
:103D50008CE092E0918380837587648757874687DC
:103D6000318B208B138B028BF58AE48AD78AC68A23
:103D7000B18EA08E938E828E8F85848F8889858F59
:103D80008989868F8A89878F8B8980A32096ECE02A
:103D90000C945725AF92BF92DF92EF92FF920F9350
:103DA0001F93CF93DF93EC017A018B01DD24403028
:103DB00081EE580780E0680780E0780711F0DD2485
:103DC000D39491E0A92EB12CEC89FD89DD2069F016
:103DD000C50108A002C0880F991F0A94E2F78083EA
:103DE00060E079E08DE390E005C0108260E874E85F
:103DF0008EE190E0A80197010E94F8242150304004
:103E000040405040569547953795279580E12030A2
:103E1000380720F0DD2011F0DD24D6CFE889F989BC
:103E20003083EA89FB89208319A2EE89FF894081CA
:103E300021E030E0C9010C8C02C0880F991F0A9460
:103E4000E2F7482B4083EE89FF894081C9010D8C40
:103E500002C0880F991F0A94E2F7482B4083EE892D
:103E6000FF894081C9010E8C02C0880F991F0A94F6
:103E7000E2F7482B4083EE89FF8980810F8C02C0D6
:103E8000220F331F0A94E2F7209528232083DF9125
:103E9000CF911F910F91FF90EF90DF90BF90AF9067
:103EA0000895DC011C96ED91FC911D97E05CFF4F9D
:103EB0002191319180819181281B390B2F733070B2
:103EC000C90108958BEA94E00E94511F892B11F0DB
:103ED0000E94201E0895DC011C96ED91FC911D9717
:103EE000E05CFF4F20813181E054F040DF01AE5BA8
:103EF000BF4F8D919C9111972817390719F42FEF17
:103F00003FEF07C08D919C91E80FF91F8081282F0A
:103F100030E0C9010895DC011C96ED91FC911D97DC
:103F2000E05CFF4F20813181E054F040DF01AE5B67
:103F3000BF4F8D919C9111972817390719F42FEFD6
:103F40003FEF10C08D919C911197E80FF91F2081D0
:103F50008D919C91119701968F73907011969C93FF
:103F60008E9330E0C9010895DC0191968C91919770
:103F7000882339F05496ED91FC915597808186FF06
:103F8000F9CF91961C920895CF93DF93EC01EE85C3
:103F9000FF85E05CFF4F20813181E054F0402F5FCE
:103FA0003F4F2F733070DF01AE5BBF4F8D919C91FF
:103FB000119728173907D1F3E05CFF4F8081918179
:103FC000E054F040E80FF91F6083EE85FF85E05C68
:103FD000FF4F31832083EE89FF89208181E090E0CB
:103FE0000F8C02C0880F991F0A94E2F7282B2083B8
:103FF00081E089A3EC89FD8980818064808381E0F0
:1040000090E0DF91CF9108958F929F92AF92BF92EF
:10401000CF92DF92EF92FF920F931F9300D000D0C8
:104020000F92EDB7FEB7319684E0ADB7BEB71196EB
:104030008C9383E0818387E0828385E0838381E0C2
:1040400084838BEA94E063E274E047E654E02DEC6D
:1040500030E00CEC10E0B8ECEB2EF12CA9ECCA2E01
:10406000D12CFAECAF2EB12CEEEC8E2E912C0E94BE
:10407000971E0F900F900F900F900F901F910F9120
:10408000FF90EF90DF90CF90BF90AF909F908F9078
:104090000895CF93DF930E942B1A85ED94E00E9440
:1040A00041210E946918C2E6DFE10E94CD0B2097F2
:1040B000E1F30E94621FF9CFFC0104C08091F1007E
:1040C000819361506623D1F7289884E68093CE04CB
:1040D00008959FB7F89487708093E9008091F2006B
:1040E0009FBF0895282F8091CF048823C1F057FFE8
:1040F0001AC015C028989093CE048091F100819346
:10410000E217F307B9F74115510539F08091F20034
:10411000882319F48BE68093E800AFBF02C04FEF0D
:104120005FEFCA010895AFB7F89427702093E900B4
:104130008091F200282F30E0241735070CF4A901F4
:10414000FB019B01240F311D94E6DACFA1E0B0E022
:10415000ECEAF0E20C944525BE016F5F7F4F41E031
:1041600050E00E947220019719F02FEF3FEF03C03B
:104170008981282F30E0C9012196E2E00C94612565
:104180002FB7F89487708093E9008091E80085FD4F
:1041900002C090E004C08091F20090E4981B2FBF11
:1041A000892F08951092E9001092D1041092D00442
:1041B0009093D3048093D2040895FF920F931F939A
:1041C000F82E142F052F4091D2045091D304212FA3
:1041D000302FC901DC01FB016EEF29C0F7FE02C0E0
:1041E000949101C090812091D0043091D104241782
:1041F0003507ACF48091E8008570E1F38091E80028
:1042000082FF03C02FEF3FEF17C09093F100C90169
:1042100001968F739070892B11F46093E8002F5FE3
:104220003F4F3093D1042093D004119731961097CB
:10423000A9F6812F902F9C01C9011F910F91FF902A
:1042400008950F931F939C01162F072F8091E8006C
:1042500082FFFCCFC901612F0E945C208BEF80930D
:10426000E800812F902F1F910F9108958093E9000E
:104270008091F200882319F08AE38093E800089582
:1042800008951092CF0481E08093D70080EA809354
:10429000D80082E189BD09B400FEFDCF61E070E085
:1042A00080E090E00E94071A80E98093D8008CE0BB
:1042B0008093E2001092E000559A209A0895A0E0C1
:1042C000B0E0E5E6F1E20C943925E82E942E852E37
:1042D0008091CF04882309F18B01242F352FC90148
:1042E000EC016AEFF62E57E0752E7E208E2D90E0C1
:1042F00040E2A42EB12CA822B9223AE3632E20E496
:10430000C22ED12CC822D9224CC08E2D0E94C02092
:10431000282F882361F4FA9419F42FEF3FEF4CC053
:1043200061E070E080E090E00E94071A3AC090E0FF
:10433000C817D9070CF42C2FC21BD1094FB7F8941A
:104340007092E900A114B10421F406C01092F100AA
:1043500021502223D9F719C0E7FC03C0F801922F9E
:1043600010C0C801322F06C0FC010196E491E09311
:10437000F10031503323C1F706C081918093F100E1
:1043800091509923D1F7020F111D8091E80085FF0C
:1043900005C0209729F4C114D10411F06092E800FF
:1043A0004FBF209709F0B1CF5D9884E68093CD048C
:1043B000292D382DC9019C01C901CDB7DEB7EEE02A
:1043C0000C9455251F920F920FB60F9211242F9324
:1043D0003F934F935F936F937F938F939F93AF938D
:1043E000BF93EF93FF938091E1001092E100982F2B
:1043F00093FF0FC01092E90081E08093EB001092D0
:10440000EC0082E38093ED001092CF0488E080936B
:10441000F00092FF28C083E00E94362182E00E94D3
:104420006920882321F085E194E00E94E71B8091B8
:10443000CD04882351F08091CD0481508093CD0428
:104440008091CD04882309F45D9A8091CE0488235D
:1044500051F08091CE0481508093CE048091CE049F
:10446000882309F4289AFF91EF91BF91AF919F9112
:104470008F917F916F915F914F913F912F910F900D
:104480000FBE0F901F901895A1E0B0E0EAE4F2E2B1
:104490000C94432519828E010F5F1F4FC8010E94A3
:1044A0000D1CC8010E94BA24898190E02196E4E0A5
:1044B0000C945F251F920F920FB60F921124CF928A
:1044C000DF92EF92FF920F932F933F934F935F935F
:1044D0006F937F938F939F93AF93BF93EF93FF93CC
:1044E000DF93CF93CDB7DEB76197DEBFCDBF10921C
:1044F000E9008091E80083FFEBC0CE01019668E0FF
:104500000E945C2082EF8093E800998197FF05C0AC
:104510008091E80080FFFCCF03C08EEF8093E8001D
:10452000292F30E0C90180769070892B09F0B1C045
:104530008A81882329F41092F1001092F100BDC005
:10454000813009F4BAC0833009F4B7C0853049F42A
:104550008091E80080FFFCCF8B8180688093E3002E
:10456000ACC0863009F06BC00C81EF80F88402305B
:1045700071F580E090E00E94D2200E94442299E0F0
:1045800079E0C72ED12CCC0EDD1EF601292F119219
:104590002A95E9F799870A8791E09E8790E8988B9A
:1045A0009AEF998B2091D0043091D104275F3F4F2F
:1045B0003C872B878D87C7010E94D22080E0B601FF
:1045C00049E050E00E94DD200E94442276C0C701ED
:1045D0000E94D220023241F482E290E00E94B22492
:1045E000892B09F46EC069C0013079F48F819885F8
:1045F000089719F481E08093D4048091D40488232F
:1046000009F063C0EDEFF1E013C0033009F059C0C9
:104610008B81882319F4EFEBF1E00AC0823019F4A2
:10462000E3ECF1E005C0813009F04BC0E5EEF1E0CC
:10463000449180E8BF0150E00E94DD203EC08730F9
:1046400009F43FC0883021F481E08093F10035C047
:10465000893099F523703070232B99F5E2E2F2E06E
:1046600091E031E026E39093E9003093EB008491F0
:104670008093EC002093ED009F5F3196953099F781
:104680008EE78093EA001092EA008B818093CF043A
:1046900014C08F8198850E94D2208D81882329F4AF
:1046A000CE0101960E94191C06C0823051F4CE0141
:1046B00001960E948323882321F08EEF8093E800E7
:1046C00007C081E28093EB0003C0EFE0F2E0B0CFDF
:1046D0006196DEBFCDBFCF91DF91FF91EF91BF918A
:1046E000AF919F918F917F916F915F914F913F918A
:1046F0002F910F91FF90EF90DF90CF900F900FBE12
:104700000F901F901895FC0191818081813A31F4BE
:10471000913089F080E0933089F40DC0813269F4E2
:104720009B3021F482818093E60105C09A3029F400
:1047300082818093E70181E0089580E00895FC0183
:1047400010820895FC01138212828CE192E0918321
:1047500080830895EF92FF920F931F938C01E62EB2
:10476000DC01ED91FC910480F581E02D0995F82E96
:10477000D801ED91FC910680F781E02DC8016E2DE6
:1047800009958F2D90E01F910F91FF90EF90089564
:1047900086ED94E00E949F2387ED94E00E94A2237F
:1047A0000895A1E0B0E0E7EDF3E20C9441258983A0
:1047B0008B017A0184E0BE016F5F7F4F41E050E0E2
:1047C0000E945F2184E4B801A7010E945F21219625
:1047D000E6E00C945D2582E048E050E00E94D123A1
:1047E0000895FC01168217821086118612861386A0
:1047F00014823496BF010E94EB230895DC016838CF
:1048000010F0685829C0E62FF0E067FF13C0E058A9
:10481000F04081E090E002C0880F991FEA95E2F72E
:10482000809514962C911497282314962C93149702
:1048300060E012C0EC55FD4F6491662319F420E04E
:1048400030E01DC067FF08C014968C9114978D7FCF
:1048500014968C9314976F77FD0190E0662321F0F6
:104860008681861709F416829F5F31969630B1F7DC
:10487000CD011496BD010E94EB2321E030E0C90177
:104880000895CF93DF93DC01683810F0685825C095
:10489000E62FF0E067FF12C0E058F04081E090E0C2
:1048A00002C0880F991FEA95E2F714962C9114978D
:1048B000282B14962C93149760E00FC0EC55FD4FF5
:1048C00064916623D9F167FF08C014968C91149700
:1048D000826014968C9314976F7716968C91169726
:1048E0008617A9F117968C911797861781F118965C
:1048F0008C911897861759F119968C9119978617EC
:1049000031F11A968C911A97861709F11B968C91A2
:104910001B978617E1F0ED01E0E0F0E09E2F8E811D
:10492000882321F4EA0FFB1F668306C09F5F319640
:104930002196E630F10591F7963049F481E090E058
:1049400013969C938E93129720E030E007C0CD0120
:104950001496BD010E94EB2321E030E0C901DF91F4
:10496000CF91089580E866E272E045E650E00E944B
:10497000DD200895FC0180818F5F808380E86BE8F3
:1049800072E049E150E00E94DD200895629FD0016D
:10499000739FF001829FE00DF11D649FE00DF11DFA
:1049A000929FF00D839FF00D749FF00D659FF00DA9
:1049B0009927729FB00DE11DF91F639FB00DE11D96
:1049C000F91FBD01CF011124089597FB092E072679
:1049D0000AD077FD04D086D006D000201AF4709556
:1049E00061957F4F0895F6F7909581959F4F0895B3
:1049F000A1E21A2EAA1BBB1BFD010DC0AA1FBB1FE3
:104A0000EE1FFF1FA217B307E407F50720F0A21B54
:104A1000B30BE40BF50B661F771F881F991F1A94C1
:104A200069F760957095809590959B01AC01BD01EB
:104A3000CF01089597FB092E05260ED057FD04D00F
:104A4000D7DF0AD0001C38F4509540953095219559
:104A50003F4F4F4F5F4F0895F6F7909580957095B3
:104A600061957F4F8F4F9F4F08952F923F924F92A6
:104A70005F926F927F928F929F92AF92BF92CF92EE
:104A8000DF92EF92FF920F931F93CF93DF93CDB7F7
:104A9000DEB7CA1BDB0B0FB6F894DEBF0FBECDBF6F
:104AA00009942A88398848885F846E847D848C8440
:104AB0009B84AA84B984C884DF80EE80FD800C8149
:104AC0001B81AA81B981CE0FD11D0FB6F894DEBF2C
:104AD0000FBECDBFED010895EE0FFF1F0590F491BD
:104AE000E02D0994AA1BBB1B51E107C0AA1FBB1FE5
:104AF000A617B70710F0A61BB70B881F991F5A956A
:104B0000A9F780959095BC01CD010895F894FFCF49
:104B100054582074696D656F757421006D6F6475EC
:104B20006C65206C6F636B65643F007363616E6ED0
:104B30006572206D6F6465004F70656E4C52536EE8
:104B400067205458207374617274696E6720002066
:104B50006F6E204857200001000000C01200001AAC
:104B6000400AA1204EA5001B1E27522C2330802571
:104B7000000005400AA1204EA50020244EA52C23AC
:104B800030004B000006400AD0009D49007B289D64
:104B9000492C233000E1000005400A4501D7DC0321
:104BA000B81E0EBF00232E48E801008A400A6001AB
:104BB000555502AD1E20000023C880250000054089
:104BC0000AA1204EA50020244EA52C23300002006F
:104BD00002000200020002000200020002000200C5
:104BE00002000200020002000200020002FF00E1D7
:104BF000000000000000010100070B0C101115005F
:104C0000160A1322312900000000BE1B6F1C5D1B19
:104C1000841B6B1BE31BE71B00000000C41F6F1C01
:104C2000511F8B1F6B1FB41F00000000AA236F1CB5
:064C30004124FE23F123E4
:00000001FF
